:1000000041C091C3B7C363C062C061C060C05FC07C
:100010005EC0D8C35CC045C676C659C058C057C07C
:1000200056C055C054C0000000000000000000038E
:1000300004060000000000000000000000010204AF
:10004000081020408001020408102001020408105A
:100050002040804004040404040404040202020258
:10006000020203030303030302020300000000383B
:10007000003500320000000000370034003100007D
:100080008F03B10611241FBECFE5D4E0DEBFCDBF84
:1000900010E0A0E6B0E0EAE8F1E102C005900D92C0
:1000A000A63DB107D9F721E0A6EDB0E001C01D9251
:1000B000A33AB207E1F710E0C2E4D0E003C0219711
:1000C000FE015BD8C034D107D1F781D75CC898CF87
:1000D00026E040E855E260E070E086E091E082D5FD
:1000E0006AE670E086E091E0B2D640EC5AEC69E84E
:1000F00076E38DED90E078D2892B31F466E770E0FD
:1001000086E091E0A4D6FFCF08956CE870E086E029
:1001100091E092D66091D6007091D7004AE050E00D
:1001200086E091E038D760E070E08DED90E0D4D2C9
:100130006DE970E08DED90E07FD66091D600709112
:10014000D7004AE050E08DED90E01FD760E08DEDE4
:1001500090E01CD18091D6009091D70001969093A9
:10016000D7008093D60068E873E180E090E09AC3FE
:10017000CF93CFB7F8948091DB0081111FC0EEE5DB
:10018000F0E08491E7E4F0E09491E82FF0E0EE0FE6
:10019000FF1FEB58FF4FA591B491EC91E92319F49F
:1001A00061E08AE02ED461E08AE0EFD36C9A6E9A27
:1001B00061E08DE0EAD361E08BE0E7D38091DB0082
:1001C0008F5F8093DB00CFBFCF910895CF93DF93F4
:1001D0001F92CDB7DEB76983DC01ED91FC910280FF
:1001E000F381E02D41E050E0BE016F5F7F4F099544
:1001F0000F90DF91CF9108950895FC011382128230
:1002000088EE93E0A0E0B0E084839583A683B78373
:1002100088EA90E09183808380E5848781E0858708
:100220008CED90E0978786878AE090E0918B808BB9
:1002300089E090E0938B828B82E090E0958B848BB9
:10024000168A178A108E118E138E128E158E148EAA
:10025000178E168E40E050E0BA01CF01B1C6EF9282
:10026000FF921F93CF93DF931F92CDB7DEB77C0130
:10027000162F60E0FC0180894983C3D3F7015485C0
:1002800035858091DA004981882399F02FB7F89459
:100290008091DA00813059F48BB78093D8009BB7F6
:1002A0008091D900809589238BBF2FBF02C02093F6
:1002B000D8005DB93EB91FB90000779BFECF8FB162
:1002C0004FB90000779BFECF1FB18091DA008823E1
:1002D00061F08FB7F8942091DA009091D800213026
:1002E00019F49BBF8FBF01C09FBF61E0F7018089F8
:1002F00088D3812F0F90DF91CF911F91FF90EF90C6
:1003000008956F7740E0ABCFCF93DF93EC0163E1CB
:10031000F8DF282F30E08A8D9B8DA901481B590BEF
:10032000CA01DF91CF910895CF93DF93EC01E8816B
:10033000F9810480F581E02D0995892B51F08A8D92
:100340009B8D01969B8F8A8F60E0CE01DADF90E073
:1003500002C08FEF9FEFDF91CF910895CF93DF938E
:10036000EC0161E0CEDF8370833051F062E1CE01B9
:10037000C8DF83FF07C048E062E9CE0170DF02C03A
:1003800081E001C080E0DF91CF9108951F93CF936A
:10039000DF93EC01162F43E861E861DF112321F0C0
:1003A00086E990E0B8D20BC062E1CE01AADF83FDFE
:1003B00002C007D2F9CF48E062E9CE0150DF81E008
:1003C00090E0DF91CF911F9108958F929F92AF920D
:1003D000BF92CF92DF92FF920F931F93CF93DF9341
:1003E0001F92CDB7DEB76C01B62E4A0162E2798367
:1003F00088DFF82E90E09C01280D391D79812F3F70
:10040000310531F028F02FEF30E04901881A990AC0
:100410000B2D172F5801A80CB91C0A151B0539F014
:10042000F80141918F0160E8C60119DFF6CF482D30
:100430004F0D62EAC60113DFC4010F90DF91CF9127
:100440001F910F91FF90DF90CF90BF90AF909F9042
:100450008F900895EF92FF921F93CF93DF931F9297
:10046000CDB7DEB77C01DC01ED91FC910480F58114
:10047000E02D0995892B81F06DE0C70142DF482FFF
:1004800060E0C70149833DDF182F49816DE8C7014E
:10049000E6DE812F90E002C08FEF9FEF0F90DF919B
:1004A000CF911F91FF90EF90089541E861E8D7CE7A
:1004B00040E861E8D4CE9F92AF92BF92CF92DF9294
:1004C000EF92FF920F931F93CF93DF93EC01DB0129
:1004D000CA014E8B5F8B688F798F6A017B01FF0C9D
:1004E000CC08DC2C76019A01AD016C2D7C2D8C2D75
:1004F0009C2D03E1F7D5A12CE8E4BE2EF8EECF2E1B
:10050000DD24D394E12CF12C00E010E0A1D5F22EF3
:10051000932E5A01162FC72ED82EE92E00E1FDD5B5
:10052000422F66E8CE019BDE2F2D392DA501612FCC
:100530007C2D8D2D9E2D08E0F0D5422F67E8CE0151
:100540008EDE4F2D68E8CE01DF91CF911F910F9184
:10055000FF90EF90DF90CF90BF90AF909F907FCEB5
:100560009C01693730F470E0CB018D9765E070E055
:1005700007C0613F38F470E0CB014E966AE070E04E
:1005800030D501C06BE16F71462F40626BE8C90145
:1005900066CE0F931F93CF93DF938C01EB016231F3
:1005A000710564F06531710514F0C4E1D0E0239762
:1005B00047E86DECC80153DE6CE80AC06230710593
:1005C00014F4C2E0D0E044E86DECC80148DE64E613
:1005D000C801C6DF4C2F4250406869E8C801DF916E
:1005E000CF911F910F913BCECF92DF92EF92FF926E
:1005F000CF93DF93EC016A017B0161E08889C5D16B
:1006000061E08889FED18A899B898F3F2FEF92070D
:1006100091F061E0BAD160E08A89F3D16AE070E0DC
:1006200080E090E03FD161E08A89EBD16AE070E040
:1006300080E090E037D19CDD62E4CE0162DE823161
:1006400019F5CE0135DFB701A601CE0134DF40E058
:100650006EE8CE0104DE40E06FE8CE0100DE6CE023
:10066000CE014FDE482F43606CE8CE01F8DD44E058
:1006700066EACE01F4DD61E170E0CE018ADFCE01F1
:1006800014DF81E090E002C080E090E0DF91CF9144
:10069000FF90EF90DF90CF900895CF93DF93EC0120
:1006A0001D8E1C8E6DE12DDE482F4E7F6DE9CE0133
:1006B000DF91CF91D4CDCF93DF93EC0181E090E037
:1006C0009D8F8C8F6DE1CE011CDE482F41606DE95E
:1006D000CE01DF91CF91C3CD0F931F93CF93DF93C3
:1006E000EC018B013BDE811113C0CE01DEDECE01B9
:1006F000012B11F0E0DF01C0D0DF40E06DE8CE015A
:10070000AEDD40E062EACE01AADD81E090E002C009
:1007100080E090E0DF91CF911F910F9108958DEDD2
:1007200090E06BCD08951F920F920FB60F92112497
:100730002F933F934F935F936F937F938F939F93E9
:10074000AF93BF93EF93FF93E0916600F091670042
:100750000995FF91EF91BF91AF919F918F917F91FB
:100760006F915F914F913F912F910F900FBE0F901E
:100770001F9018951F920F920FB60F9211242F936E
:100780003F934F935F936F937F938F939F93AF9319
:10079000BF93EF93FF93E0916800F0916900099592
:1007A000FF91EF91BF91AF919F918F917F916F9149
:1007B0005F914F913F912F910F900FBE0F901F901F
:1007C000189508951F920F920FB60F9211242F9330
:1007D0003F938F939F93AF93BF938091FE0090912F
:1007E000FF00A0910001B09101013091FD0026E0D1
:1007F000230F2D3720F40296A11DB11D05C029E855
:10080000230F0396A11DB11D2093FD008093FE00D0
:100810009093FF00A0930001B09301018091020129
:1008200090910301A0910401B09105010196A11DD1
:10083000B11D8093020190930301A0930401B09332
:100840000501BF91AF919F918F913F912F910F9093
:100850000FBE0F901F9018953FB7F894809102013A
:1008600090910301A0910401B091050122B708B64F
:1008700000FE05C02F3F19F00196A11DB11D3FBF1D
:10088000BA2FA92F982F8827820F911DA11DB11D66
:10089000BC01CD0143E0660F771F881F991F4A9561
:1008A000D1F708958F929F92AF92BF92CF92DF922D
:1008B000EF92FF926B017C01CFDF4B015C01C11411
:1008C000D104E104F104F1F07CDFC6DFDC01CB01EF
:1008D00088199909AA09BB09883E9340A105B10569
:1008E00070F321E0C21AD108E108F10888EE880E01
:1008F00083E0981EA11CB11CC114D104E104F104D1
:1009000021F7DDCFFF90EF90DF90CF90BF90AF90B9
:100910009F908F9008958330910528F0880F991F3C
:1009200004970197F1F70895789483B7826083BFA5
:1009300083B7816083BF89B7816089BF1EBC8EB5D4
:1009400082608EBD8EB581608EBD8FB581608FBD9A
:1009500085B5846085BD85B5806485BD329A319A40
:100960003098379A1AB80895843039F0863049F0B3
:10097000833051F48FB58F7702C08FB58F7D8FBDD7
:10098000089585B58F7D85BD0895CF93DF9390E061
:10099000FC01E35CFF4F2491FC01EC5AFF4F849172
:1009A000882361F190E0880F991FFC01EB58FF4FFD
:1009B000C591D491FC01E559FF4FA591B491611106
:1009C00009C09FB7F8948881209582238883EC9191
:1009D0002E230BC0623061F49FB7F8943881822FC8
:1009E000809583238883EC912E2B2C939FBF06C088
:1009F0008FB7F894E8812E2B28838FBFDF91CF919A
:100A000008951F93CF93DF93282F30E0F901EA5D1B
:100A1000FF4F8491F901E35CFF4FD491F901EC5A47
:100A2000FF4FC491CC23C1F0162F81119DDFEC2F15
:100A3000F0E0EE0FFF1FE559FF4FA591B4918FB77E
:100A4000F894111105C09C91ED2FE095E92302C0A7
:100A5000EC91ED2BEC938FBFDF91CF911F91089517
:100A6000FC01918D228D892F90E0805C9F4F821B2D
:100A700091098F7399270895FC01918D828D9817A4
:100A800031F0828DE80FF11D858D90E008958FEF94
:100A90009FEF0895FC01918D828D981761F0828DF2
:100AA000DF01A80FB11D5D968C91928D9F5F9F73A2
:100AB000928F90E008958FEF9FEF089588EA96E077
:100AC000892B39F080E090E0892B19F041D1811118
:100AD00097CA0895FC01848DDF01A80FB11DA35AA8
:100AE000BF4F2C91848D90E001968F739927848F4E
:100AF000A689B7892C93A089B1898C9180648C9345
:100B0000938D848D981306C00288F389E02D80812F
:100B10008F7D80830895CF93DF93EC01888D8823A8
:100B2000C1F0EA89FB89808185FD05C0A889B98962
:100B30008C9186FD0EC00FB607FCF5CF808185FF36
:100B4000F2CFA889B9898C9185FFEDCFCE01C2DFA4
:100B5000E8CFDF91CF910895EF92FF920F931F930B
:100B6000CF93DF93EC0181E0888F9B8D8C8D981360
:100B700005C0E889F989808185FD23C0F62E0B8D9B
:100B800010E00F5F1F4F0F731127E02E8C8DE812BE
:100B90000BC00FB607FCFACFE889F989808185FF81
:100BA000F5CFCE0197DFF2CF8B8DFE01E80FF11D5F
:100BB000E35AFF4FF0820B8FEA89FB8980818062C4
:100BC00007C0EE89FF896083E889F98980818064A4
:100BD000808381E090E0DF91CF911F910F91FF9092
:100BE000EF900895CF92DF92EF92FF921F93CF93F1
:100BF000DF93EC016A017B01122F60E874E88EE15B
:100C000090E0A701960100D2DA01C9010197A1097C
:100C1000B109B695A79597958795AC01E889F989AB
:100C200082E08083411580E15807A0F0E889F989C6
:100C3000108260E472E48FE090E0A7019601E4D1B5
:100C4000BA01A90141505109610971097695679569
:100C500057954795EC85FD855083EE85FF8540834C
:100C6000188E1068EC89FD891083EA89FB898081E0
:100C700080618083EA89FB89808188608083EA893A
:100C8000FB89808180688083EA89FB8980818F7DF0
:100C90008083DF91CF911F91FF90EF90DF90CF90F5
:100CA00008951F920F920FB60F9211242F938F93D6
:100CB0009F93EF93FF93E0911601F09117018081CC
:100CC000E0911C01F0911D0182FD12C09081809184
:100CD0001F018F5F8F7320912001821751F0E091E7
:100CE0001F01F0E0EA5FFE4F958F80931F0101C066
:100CF0008081FF91EF919F918F912F910F900FBE67
:100D00000F901F9018951F920F920FB60F921124FB
:100D10002F933F934F935F936F937F938F939F9303
:100D2000AF93BF93EF93FF9386E091E0D3DEFF9103
:100D3000EF91BF91AF919F918F917F916F915F9153
:100D40004F913F912F910F900FBE0F901F901895CC
:100D500086E091E085DE21E0892B09F420E0822FF6
:100D60000895E6E0F1E01382128288EE93E0A0E0BD
:100D7000B0E084839583A683B78388EB90E091836A
:100D8000808380E490E09587848729E230E037878C
:100D900026872BE230E0318B208B2AE230E0338B48
:100DA000228B958B848B8CE290E0978B868B118EB7
:100DB000128E138E148E0895CF92DF92EF92FF92CF
:100DC0000F931F93CF93DF936C017A018B01C0E0E7
:100DD000D0E0CE15DF0589F0D8016D918D01D601E7
:100DE000ED91FC910190F081E02DC6010995892BD0
:100DF00011F47E0102C02196ECCFC701DF91CF91A3
:100E00001F910F91FF90EF90DF90CF9008956115A3
:100E1000710579F0FB0101900020E9F73197AF01EE
:100E2000461B570BDC01ED91FC910280F381E02D14
:100E3000099480E090E00895EACFDC01ED91FC9107
:100E40000190F081E02D099464EC70E0E0CF0F9305
:100E50001F93CF93DF93EC01DADF8C01CE01F4DF37
:100E6000800F911FDF91CF911F910F9108954F92A5
:100E70005F926F927F92EF92FF920F931F93CF93A7
:100E8000DF93CDB7DEB7A1970FB6F894DEBF0FBEE4
:100E9000CDBF7C01FA01CB0119A2223008F42AE06F
:100EA0008E010F5D1F4F422E512C612C712CBF0102
:100EB000A3019201A9D0F901CA01015011096A30B8
:100EC00014F4605D01C0695CD8016C93232B242B62
:100ED000252B69F7B801C7019ADFA1960FB6F894E0
:100EE000DEBF0FBECDBFDF91CF911F910F91FF905D
:100EF000EF907F906F905F904F900895CF92DF9228
:100F0000EF92FF920F931F93CF93DF93EC016A014F
:100F10007B012115310579F4E881F9810190F08197
:100F2000E02D642FDF91CF911F910F91FF90EF90F3
:100F3000DF90CF9009942A303105D9F477FF18C09B
:100F40006DE27BDF8C0144275527BA014C195D09FE
:100F50006E097F092AE0CE018ADF800F911FDF91A1
:100F6000CF911F910F91FF90EF90DF90CF90089558
:100F70002AE0B701A601CE01DF91CF911F910F9119
:100F8000FF90EF90DF90CF9072CF9A01AB01770F77
:100F9000660B770BB3CF0F931F93CF93DF93EC01C7
:100FA0009A01AB01770F660B770BA8DF8C01CE019E
:100FB0004BDF800F911FDF91CF911F910F9108950B
:100FC000FC01448355836683778308950895ACDCE0
:100FD000FDDF7ED8CEE5D5E098D82097E9F36EDD29
:100FE000FBCF97FB072E16F4009406D077FD08D0B0
:100FF000B0D007FC05D03EF4909581959F4F0895A1
:10100000709561957F4F0895A1E21A2EAA1BBB1B14
:10101000FD010DC0AA1FBB1FEE1FFF1FA217B307C4
:10102000E407F50720F0A21BB30BE40BF50B661FDA
:10103000771F881F991F1A9469F76095709580959E
:1010400090959B01AC01BD01CF010895689401C04A
:10105000E8948F929F92CF93DF9305D0DF91CF9149
:101060009F908F90089588249924F401E401B0E4BE
:101070001B2ED4019D158E049F04E007F10738F460
:10108000FC014B01CA01B901AD019E011694220F6A
:10109000331F441F551F661F771F881F991F881C09
:1010A000991CEE1FFF1FCC1FDD1FAA1FBB1F8A1438
:1010B0009B04EC05FD05CE05DF05A007B10748F050
:1010C0008A189B08EC09FD09CE09DF09A00BB10BBA
:1010D00021601A94E1F62EF49401AF01BE01CD0116
:1010E000000C08950F93083090F0982F872F762FDB
:1010F000652F542F432F322F22270850F4CF220F71
:10110000331F441F551F661F771F881F991F0A959D
:10111000B2F70F91089597FB10F8169400080F93FB
:10112000083098F00850232F342F452F562F672F63
:10113000782F892F902DF4CF0594979587957795E3
:10114000679557954795379527950A95AAF70F9173
:101150000895AA1BBB1B51E107C0AA1FBB1FA617FE
:10116000B70710F0A61BB70B881F991F5A95A9F750
:1011700080959095BC01CD010895EE0FFF1F05905D
:0A118000F491E02D0994F894FFCFDC
:10118A000000A3018000920392034C6F5261205326
:10119A00656E646572005374617274696E67204C7F
:1011AA006F5261206661696C6564210053656E64E3
:1011BA00696E67207061636B65743A200068656CBC
:1011CA006C6F200000000000E600E5018401940134
:1011DA002A02FC0000000000AC05DC0630054A05C6
:1011EA003C058B050D0A006E616E00696E66006F24
:0611FA007666002E0000E5
:00000001FF
